:10000000370101007128A948730000008280148123
:10001000988133E6E60009C685050505E389E6FE15
:1000200013351600828052B82A84592C2A94492C00
:10003000E36F85FE52BE8AB8952C25C11304400695
:1000400093045006130940079309300619A0B92CF0
:1000500029C5014549240808C1450A86C146A12C85
:1000600003450101E31585FE03451101E31195FEEA
:1000700003452101E31D25FD03453101E31995FCED
:1000800003454101E31535FD03455101E31125FD0C
:10009000034561014DFD05458ABE05452D2C8ABCF1
:1000A000FAB813058031F5221305E032DD2213047E
:1000B0000035930560352285ED221309A03593059F
:1000C000F0354A85F92A130A303693058036528571
:1000D000C92AED2A930B4006130C5006930D4007D6
:1000E00093043006930C203F130DE03F930A104019
:1000F0001305B036792A0545F92A13051037512A18
:10010000752221C50145C12A0808C1450A86C14694
:100110005D2203450101E31575FF03451101E3115C
:1001200085FF03452101E31DB5FD03453101E319B9
:1001300085FD03454101E31595FC03455101E3119C
:10014000B5FD034561014DFD21A0054569224DBF67
:10015000130520383D2A0145BD2A22859305303AF2
:1001600089221305A03A3522A12A93092500892A5C
:10017000E36F35FF4A859305903B25221305C03B6D
:10018000092A3D2A93092500252AE36F35FF228598
:100190009305603C39221305A03CE52815229309FC
:1001A0003500392AE36F35FF52859305603DD52828
:1001B0001305B03DF9282922930945001122E36F68
:1001C00035FF4A859305F035E9281305703ED120A7
:1001D000F528BD4909A80545FD280145ED28FD196B
:1001E00013F5F90F3DC913FBF90F66855D205A859C
:1001F00069286A857928E920130B1500D120E36F5F
:1002000065FF6D2069D90145F9200808C1450A86B6
:10021000C146552003450101E31575FF0345110152
:10022000E31185FF03452101E31DB5FD03453101C0
:10023000E31985FD03454101E31595FC0345510193
:10024000E311B5FD034561014DFD71204120568547
:100250008920E14913F5F90F59F513056041152877
:100260005285930580363528130510421D208928B4
:1002700093092500B120E36F35FF22859305603592
:100280000D201305B0423120A5B58548730000004C
:1002900082809148730000008280AD4873000000A6
:1002A0008280930810087300000082809308500831
:1002B0007300000082809308700873000000828041
:1002C000732510C08280732500C082809308600867
:1002D0007300000082800589F32200809392024817
:1002E000B3E2A20073900280828095487300000000
:1002F000828093080008730000008280A148730088
:100300000000828093083008730000008280930808
:1003100040087300000082804445205261696C727D
:100320006F61642043726F7373696E670A00666F52
:1003300072205256436F6E74726F6C6C65720A490C
:100340006E697469616C697A696E672048570A0042
:100350006C69676874004F46460062656C6C006F9C
:10036000666600676174650075700049646C650AB3
:10037000004C696768747765696768743A204F6EE6
:100380000A00547261696E20646574656374656403
:100390000A4C696768747765696768743A204F66C4
:1003A000660A0059454C4C4F57004C696768743ACF
:1003B0002059656C6C6F770A006F6E0042656C6C3B
:1003C0003A204F6E0A00524544004C696768743AFF
:1003D000205265640A00646F776E00476174653A65
:1003E00020446F776E0A0042656C6C3A204F666657
:1003F0000A0054696D656F757420696E2000730A78
:100400000054696D6520726573657420627920748B
:100410007261696E0A0054696D6564206F75740AB3
:1004200000476174653A2055700A004C696768742A
:070430003A204F66660A0046
:00000001FF
